:100000000BC018951895189518951895189518956A
:1000100018951895189518958FED8DBFC0ECE4EBE9
:100020004E2EDD275D2EEEE7F0E0A0E6B0E088275B
:100030008D933197E9F784B7082E877F84BF8FE1CE
:1000400081BD87E081BD63D166248FEF8ABB8FE0DD
:1000500087BB80E08BBB80E088BB83E886B980E803
:1000600087B98CE09CD139D1ECECF7E030D1E2E0FB
:10007000F0E044D132D18FE714E03ED1ECEDF7E06F
:1000800026D100916E000A3008F003C0E2EEF7E0DE
:100090001ED1ACE9B0E0EEE6F0E038D310D1E4EEEA
:1000A000F7E015D1ACE9B0E0EFE6F0E02FD307D1EF
:1000B0008FE71CE021D1E6EEF7E009D18FEB14E0E9
:1000C0001BD1EAEEF7E003D1ACE9B0E0E0E7F0E005
:1000D0001DD3F5D0E4EEF7E0FAD0A1E70D911C9125
:1000E0000A3050E0150708F003C0E0EFF7E0EFD06A
:1000F000ACE9B0E0E1E7F0E0FAD2E1D08FEB1CE050
:10010000FBD0E2EFF7E0E3D0A4E78C9187FB8827F0
:1001100080F9809580FBA4E78C9187F98C93A4E704
:100120008C9187FB0EF404C087E08093750003C0B8
:1001300089E18093750088EC90E05DD1379AEF9368
:10014000FF93E5E1F0E04BD1FF91EF9107B1007E25
:10015000A5E78C9190E0890F082707B95BD1A0E64D
:100160008D939C933798E0E6F0E0D190E080FF24F7
:100170000027BBD1A2E6EAD1ECEAF7E08BD2E2E6B7
:10018000F0E08FD1F5D1EDE0A2E60AD3A4E78C919F
:1001900087FB0EF432C0E0EBF7E07CD2E2E6F0E061
:1001A00080D1E6D1EDE0A2E6FBD2E2E6F0E03BD181
:1001B000AEE6DC92EEE6F0E0D080EE24FF240027ED
:1001C00094D1A6E6C3D1E6E6F0E070D1E2E6F0E035
:1001D00068D1FFD1EDE0A2E6E3D2E4EBF7E05AD23A
:1001E000E2E6F0E05ED1C4D1EDE0A2E6D9D2E2E6EB
:1001F000F0E019D1AFE6DC9261C0E2E6F0E051D167
:10020000E8EBF7E047D24FD208F00AC0ECEBF7E09A
:1002100041D2E2E6F0E045D1ABD1EDE0AAE6C0D2B2
:10022000E2E6F0E03ED1E8EBF7E034D23CD208F46D
:100230000AC0E0ECF7E02ED2E2E6F0E032D198D14D
:10024000EDE0AAE6ADD2EAE6F0E0EDD0A0E7DC9280
:10025000E0E7F0E0D080EE24FF24002746D1A6E6B8
:1002600075D1E6E6F0E022D1EAE6F0E01AD1B1D1AC
:10027000EDE0AAE695D2E4ECF7E00CD2EAE6F0E095
:1002800010D176D1EDE0AAE68BD2EAE6F0E0CBD051
:10029000A1E7DD92EC92E2E6F0E003D1E8ECF7E0D2
:1002A000F9D101D210F009F001C008C081E08093BB
:1002B000700082E390E0A1E78D939C93DCCEACE9E3
:1002C000B0E08D91882311F064D0FBCF0895DED18A
:1002D000802D11F05ED0FBCF089581E060D014D066
:1002E00080E85DC08FE7213039F08FEB223021F0BC
:1002F0008FE8233009F08FEC810F51C088EE93E036
:100300007AD03197D9F7089583E0992774C08AEF9E
:1003100090E071D0B89AB99ABA9ABB9AD49AD59A01
:10032000DD9885E090E067D0DC98C098C198C29ACB
:10033000C39ADC9AEF93FF93E5E1F0E050D0FF9190
:10034000EF91DC9855D0DC9AEF93FF93E5E1F0E074
:1003500046D0FF91EF91DC984BD0DC9AEF93FF935E
:10036000E5E1F0E03CD0FF91EF91DC9841D0C398FB
:10037000DC9AEF93FF93E5E1F0E031D0FF91EF914C
:10038000DC9836D088E20BD08EE009D086E007D02A
:100390000895DD9A829505D004D02AD00895DD987D
:1003A000F9CF859510F4C39A01C0C398859510F4D0
:1003B000C29A01C0C298859510F4C19A01C0C19833
:1003C000859510F4C09A01C0C098DC9AEF93FF9312
:1003D000E5E1F0E004D0FF91EF91DC9808953197CA
:1003E000F1F70895689462F80895E89462F8089522
:1003F00081E090E000C0EF93FF93EE27E82BE92B1C
:1004000031F0EAEFF0E03197F1F70197D1F7FF9182
:10041000EF910895369A3699FECF369A3699FECFE7
:1004200084B195B108953DD0992711278F2D880F5C
:1004300080E8F82A802F881F08F41FEF41F08F57BB
:10044000082F07FD04C0003240F08FEF01C088275D
:10045000982FD82EE82EF82E09C08FE1801B082F88
:10046000F694E794D79497950A95D1F7112351F014
:100470009095D094E094F09481E0980F8827D81E4E
:10048000E81EF81E0F2DFE2CED2CD92E0895D094C9
:10049000E094F09491E0D90E9927E91EF91E109589
:1004A0000895D190E190F1900191089521913191B9
:1004B000419151910895102F90E8FF0C001F0927DA
:1004C000990FF7941078652F90E8440F551F59271E
:1004D000990F4795607800380895FF0C90E89027B1
:1004E000110F9795F794092F0895102FBD2CDE2C2E
:1004F000EF2CF02E11234AF4B094D094E094F094B1
:100500009FEFB91AD90AE90AF90A0EE1FF2039F476
:10051000FE2CED2CDB2CBB240850C2F723C032F09C
:100520000A95BB0CDD1CEE1CFF1CF9CF01D0D5CF0A
:10053000B7FE089590E8B91611F4D0FE08959FEF24
:10054000D91AE90AF90A09F403950895DD92ED92A2
:10055000FD920C9308959FE7092FF92A9FEFD92E5A
:10056000E92E0895DD24EE24FF24002711270895A5
:10057000A2DFC1F35038B1F3162700585058089441
:10058000051F12F418F4E7CF08F0ECCF0AD0FF20D3
:100590002AF0BB0CDD1CEE1CFF1C9FCF0F5FDBF2B3
:1005A0009CCF9F929924AA24BB24992788E1990C77
:1005B000AA1CBB1CDD1CEE1CFF1C30F4920EA31EFB
:1005C000B41ED91EE91EF91E8A9589F79F900895D9
:1005D0006DDF71DF503829F090E869270CC00AF010
:1005E00045D07BCF5FE322273327442701C05EDF5E
:1005F00062DF5038B1F3003899F3902F951B8BF3DD
:1006000012F434D0FACF983118F022273327442738
:10061000983028F0232F342F44279850F9CF99236E
:1006200029F04695379527959A95D9F7912F9627D2
:1006300042F014D0B0F6F794E794D7940F5F8BF69E
:100640008ACF10D051F008F422DFFF2052F2DD0CE7
:10065000EE1CFF1C0150CBF77ECF84CFD20EE31EE1
:10066000F41E0895D21AE30AF40A0895DF92EF9275
:10067000FF920F931F93D22EE32EF42E052F162FE9
:100680006F915F914F913F912F910895C895319649
:1006900000200895FBDF202DF9DF302DF7DF402DFE
:1006A000F5DF502D089507FB00680EF40F7757FB18
:1006B00050680EF45F7707FD02C057FF05C0D216E1
:1006C000E306F406050708952D153E054F0550076E
:1006D0000895000F111F221F331F089500951095D4
:1006E000209530950F5F1F4F2F4F3F4F0895019179
:1006F00010810EC001911191219130810BC00191A7
:10070000108117FF05C03FEF2FEF04C000811127B4
:100710002227332737FF03C0E1DF8DE28D93CF938C
:10072000DF93CF92DF92EF92AA24BB24CC24DD2466
:10073000EE2440E2CAE0DD2755E093E38881890F8B
:1007400087FD9F7083FD907F891B89935A95A9F738
:10075000C0DFAA1CBB1CCC1CDD1CEE1C4A9551F74B
:10076000E894EFE0FF2782910ED0EB30E0F71EF027
:1007700068948A2D0CD088278D93EF90DF90CF90CE
:10078000DF91CF910895982F829501D0892F8F7096
:10079000805D26F0803309F4089568948D93089560
:1007A00094E081918D939A95E1F708951283803EAC
:1007B000295C0F3E00002041000040404260653C43
:1007C0005839343C0000C842000007435757572EA1
:1007D0004156522E344D472E434F4D0055203D205B
:1007E000000020002E002056000049203D2000007F
:0607F00030002041000072
:00000001FF
